:020000040000FA
:020000000528D1
:08000800F62883018B0185013C
:100010000730990083162830850070308F008830B3
:1000200081000C1083128B12013090000B178B177C
:10003000C701C4016F20BB20851923280130C706E2
:10004000AB20C830E52044183628851A1C28C80182
:10005000C901CA01CB01C501C60144143830810071
:100060002430C0005430C1008B163A28851E692800
:10007000451C1C2807304B1C480885004B08031DF5
:100080004B280310C50D4A08031D4B28C50D490810
:10009000031D4B28C50DC608031954289A20FA30B1
:1000A000E520C60B4E286728C50C031C5A28471CA0
:1000B0008C206728C50C031C5F2893206728C50C7B
:1000C000031C6428A02067289E204808C600C5019C
:1000D0001C288B12C40107308500B6201C2875200F
:1000E000812075208120752008000630CC004C0846
:1000F000063C8500F42007308500F420CC0B7728DF
:1001000008000630CC004C038500F4200730850041
:10011000F420CC0B83280800F630C2000930C3005D
:100120006430DD200800F830C2008930C30064303C
:10013000DD2008008C20F22093200800A020F2206F
:100140009320F22093200800F130C2001230C30047
:100150006430DD200800A420F220A4200800F13043
:10016000C2001230C300FA30DD200800A420643041
:10017000E520AF200800F130C2001230C300C830C3
:10018000DD20F420F430C2002630C300C830DD206A
:10019000F420F630C2000930C300C830DD20F4205E
:1001A000F830C2008930C300C830DD20F830C2000A
:1001B0008930C300C830DD20080083160C14831278
:1001C000E52083160C1083120800CE00DD30CF002E
:1001D000E928EA28EB28CF0BE828EE28EF28CE0BF9
:1001E000E62808001E30E5283230E528F000030834
:1001F000F10083120B19FF280C182B2932290B113F
:10020000383081000130C10203190A29031832294C
:10021000C0023229C008031D32292430C0005430E6
:10022000C1004514CB0A0A304B02031C3229CB0112
:10023000CA0A06304A02031C3229CA01C90A0A3016
:100240004902031C3229C901C80A06304802031CAE
:100250003229C80132290C1042088F0043088E0051
:0E0260001030850671088300F00E700E090044
:02400E00C43CB0
:00000001FF
